:020000040000FA
:0408000063EF09F0A9
:1008100003B26EEF05F0F2B48CEF05F09EB094EFEA
:1008200005F09EB29CEF05F0F2A81AEF04F0F2B2C8
:100830001CEF04F012EF09F0CD90F2929EA026EF8B
:1008400004F00101533F26EF04F0542BB2C1B6F17E
:10085000B3C1B7F1B4C1B8F1B5C1B9F1AEC1B2F12C
:10086000AFC1B3F1B0C1B4F1B1C1B5F1AAC1AEF13C
:10087000ABC1AFF1ACC1B0F1ADC1B1F1A6C1AAF14C
:10088000A7C1ABF1A8C1ACF1A9C1ADF1A2C1A6F15C
:10089000A3C1A7F1A4C1A8F1A5C1A9F19EC1A2F16C
:1008A0009FC1A3F1A0C1A4F1A1C1A5F19AC19EF17C
:1008B0009BC19FF19CC1A0F19DC1A1F1CECF9AF146
:1008C000CFCF9BF153C19CF154C19DF1CF6ACE6A49
:1008D0000101536B546B9E90CD800FBC0F8E0FBAED
:1008E00075EF04F00F8A12EF09F013880F8C0FBE1A
:1008F000B2EF04F09AC19EF19BC19FF19CC1A0F19F
:100900009DC1A1F19EC1A2F19FC1A3F1A0C1A4F11B
:10091000A1C1A5F1A2C1A6F1A3C1A7F1A4C1A8F1EB
:10092000A5C1A9F1A6C1AAF1A7C1ABF1A8C1ACF1BB
:10093000A9C1ADF1AAC1AEF1ABC1AFF1ACC1B0F18B
:10094000ADC1B1F1AEC1B2F1AFC1B3F1B0C1B4F15B
:10095000B1C1B5F1B2C1B6F1B3C1B7F1B4C1B8F12B
:10096000B5C1B9F101015E6B5F6B606B616B9A5150
:100970005E279B515F239C5160239D5161239E51B3
:100980005E279F515F23A0516023A1516123A25193
:100990005E27A3515F23A4516023A5516123A65173
:1009A0005E27A7515F23A8516023A9516123AA5153
:1009B0005E27AB515F23AC516023AD516123AE5133
:1009C0005E27AF515F23B0516023B1516123B25113
:1009D0005E27B3515F23B4516023B5516123B651F3
:1009E0005E27B7515F23B8516023B9516123D89076
:1009F0000101613360335F335E33D89001016133AD
:100A000060335F335E33D8900101613360335F330D
:100A10005E3300C10CF101C10DF102C10EF103C141
:100A20000FF104C110F105C111F106C112F107C1A6
:100A300013F108C114F109C115F10AC116F10BC176
:100A400017F134C135F111B831EF05F00101620E33
:100A5000046F010E056F000E066F000E076F3AEF70
:100A600005F00101A70E046F020E056F000E066F60
:100A7000000E076F5EC100F15FC101F160C102F1BC
:100A800061C103F1C4EC22F003BF04D01CBE02D04C
:100A90001CA0108C11A052EF05F010BA52EF05F017
:100AA0000F80108A0CC100F10DC101F10EC102F1DD
:100AB0000FC103F110C104F111C105F112C106F11A
:100AC00013C107F114C108F115C109F116C10AF1EA
:100AD00017C10BF135C134F112EF09F00392ABB23B
:100AE000AB98AB88030103EE00F080517F0BE92641
:100AF00004C0EFFF802B8151805D700BD8A48B82E6
:100B000000008051815D700BD8A48B9281518019B7
:100B1000D8B4079012EF09F0F2940101453F12EFAB
:100B200009F0462B12EF09F09E900101533F12EF9E
:100B300009F0542B12EF09F09E9213A0C6EF05F0B6
:100B400001015E6B5F6B606B616B626B636B646B0F
:100B5000656B666B676B686B696B536B546BCF6AC5
:100B6000CE6A0F9A0F9C0F9E0101476B486B496B31
:100B70004A6B4B6B4C6B4D6B4E6B4F6B506B516BB1
:100B8000526B456B466BD76AD66A139011B83BEF30
:100B900007F08BB4D3EF05F010ACD3EF05F08B84E6
:100BA000109CD4EF05F08B94C3CF55F1C4CF56F110
:100BB000C28207B443EF06F047C14BF148C14CF184
:100BC00049C14DF14AC14EF15EC162F15FC163F1AD
:100BD00060C164F161C165F113A8F1EF05F0138CF8
:100BE00013989AC1BAF19BC1BBF19CC1BCF19DC1E4
:100BF000BDF19EC1BEF19FC1BFF1A0C1C0F1A1C1B5
:100C0000C1F1A2C1C2F1A3C1C3F1A4C1C4F1A5C184
:100C1000C5F1A6C1C6F1A7C1C7F1A8C1C8F1A9C154
:100C2000C9F1AAC1CAF1ABC1CBF1ACC1CCF1ADC124
:100C3000CDF1AEC1CEF1AFC1CFF1B0C1D0F1B1C1F4
:100C4000D1F1B2C1D2F1B3C1D3F1B4C1D4F1B5C1C4
:100C5000D5F1B6C1D6F1B7C1D7F1B8C1D8F1B9C194
:100C6000D9F1010155515B2756515C23E86A5D2398
:100C70000E2E43EF06F05CC157F15DC158F15B6B7E
:100C80005C6B5D6B078E0201002F12EF09F03C0ECA
:100C9000006F1D50E00BE00AE86612881BBE02D010
:100CA0001BB4108E00C10CF101C10DF102C10EF197
:100CB00003C10FF104C110F105C111F106C112F118
:100CC00007C113F108C114F109C115F10AC116F1E8
:100CD0000BC117F134C135F101018E6777EF06F0D2
:100CE0008F6777EF06F0906777EF06F091677BEFFD
:100CF00006F0ACEF06F092C100F193C101F194C18E
:100D000002F195C103F10101010E046F000E056FA0
:100D1000000E066F000E076FC4EC22F000C192F1C6
:100D200001C193F102C194F103C195F10101006782
:100D3000A1EF06F00167A1EF06F00267A1EF06F050
:100D40000367ACEF06F08EC192F18FC193F190C1B1
:100D500094F191C195F10F80D57ED5BE6ED0D6CFDE
:100D600047F1D7CF48F145C149F1E86AE8CF4AF1E8
:100D7000138A1CBE02D01CA0108C109047C100F139
:100D800048C101F149C102F14AC103F101010A0E52
:100D9000046F000E056F000E066F000E076FC4ECA7
:100DA00022F003AF1080010154A7E3EF06F00F9A81
:100DB0000F9C0F9E0101000E5E6F600E5F6F3D0E77
:100DC000606F080E616F010147BFF3EF06F04867DF
:100DD000F3EF06F04967F3EF06F04A67F3EF06F02A
:100DE000F28818EF07F0F2985E6B5F6B606B616BD7
:100DF0009A6B9B6B9C6B9D6B9E6B9F6BA06BA16BAF
:100E0000A26BA36BA46BA56BA66BA76BA86BA96B5E
:100E1000AA6BAB6BAC6BAD6BAE6BAF6BB06BB16B0E
:100E2000B26BB36BB46BB56BB66BB76BB86BB96BBE
:100E3000D76AD66A0101456B466B0CC100F10DC142
:100E400001F10EC102F10FC103F110C104F111C192
:100E500005F112C106F113C107F114C108F115C162
:100E600009F116C10AF117C10BF135C134F112EFC6
:100E700009F012EF09F00201002F96EF08F0D59E5D
:100E8000D6CF47F1D7CF48F145C149F1E86AE8CF5D
:100E90004AF1138AD76AD66A0101456B466BD58E33
:100EA0001D50E00BE00AE86612881BBE02D01BB49E
:100EB000108E1AAE1F8C00C10CF101C10DF102C1E0
:100EC0000EF103C10FF104C110F105C111F106C10A
:100ED00012F107C113F108C114F109C115F10AC1DA
:100EE00016F10BC117F134C135F10FA0109A11B8EA
:100EF00085EF07F00101620E046F010E056F000E11
:100F0000066F000E076F8EEF07F00101A70E046F4A
:100F1000020E056F000E066F000E076F47C100F14D
:100F200048C101F149C102F14AC103F1C4EC22F008
:100F300003BFA1EF07F01CBE02D01CA0108C11B0A3
:100F40000F800CC100F10DC101F10EC102F10FC102
:100F500003F110C104F111C105F112C106F113C171
:100F600007F114C108F115C109F116C10AF117C141
:100F70000BF135C134F102013C0E006F00C10CF1E0
:100F800001C10DF102C10EF103C10FF104C110F155
:100F900005C111F106C112F107C113F108C114F125
:100FA00009C115F10AC116F10BC117F134C135F1B0
:100FB00001018E67E3EF07F08F67E3EF07F09067BB
:100FC000E3EF07F09167E7EF07F018EF08F092C141
:100FD00000F193C101F194C102F195C103F1010146
:100FE000010E046F000E056F000E066F000E076FF6
:100FF000C4EC22F000C192F101C193F102C194F15D
:1010000003C195F1010100670DEF08F001670DEFD5
:1010100008F002670DEF08F0036718EF08F08EC1C3
:1010200092F18FC193F190C194F191C195F10F802C
:10103000109047C100F148C101F149C102F14AC114
:1010400003F101010A0E046F000E056F000E066F1A
:10105000000E076FC4EC22F003AF1080010154A70B
:101060003EEF08F00F9A0F9C0F9E0101000E5E6F7D
:10107000600E5F6F3D0E606F080E616F47C100F13B
:1010800048C101F149C102F14AC103F10101140E45
:10109000046F050E056F000E066F000E076FC4EC9F
:1010A00022F003AF57EF08F0F2887CEF08F0F298D7
:1010B0005E6B5F6B606B616B9A6B9B6B9C6B9D6BEC
:1010C0009E6B9F6BA06BA16BA26BA36BA46BA56BBC
:1010D000A66BA76BA86BA96BAA6BAB6BAC6BAD6B6C
:1010E000AE6BAF6BB06BB16BB26BB36BB46BB56B1C
:1010F000B66BB76BB86BB96B0CC100F10DC101F1E8
:101100000EC102F10FC103F110C104F111C105F1CB
:1011100012C106F113C107F114C108F115C109F19B
:1011200016C10AF117C10BF135C134F18BB4A0EF30
:1011300008F010ACA0EF08F08B84109CA1EF08F031
:101140008B94C3CF55F1C4CF56F1C28207B410EFD0
:1011500009F047C14BF148C14CF149C14DF14AC1B9
:101160004EF15EC162F15FC163F160C164F161C1C2
:1011700065F113A8BEEF08F0138C13989AC1BAF169
:101180009BC1BBF19CC1BCF19DC1BDF19EC1BEF133
:101190009FC1BFF1A0C1C0F1A1C1C1F1A2C1C2F103
:1011A000A3C1C3F1A4C1C4F1A5C1C5F1A6C1C6F1D3
:1011B000A7C1C7F1A8C1C8F1A9C1C9F1AAC1CAF1A3
:1011C000ABC1CBF1ACC1CCF1ADC1CDF1AEC1CEF173
:1011D000AFC1CFF1B0C1D0F1B1C1D1F1B2C1D2F143
:1011E000B3C1D3F1B4C1D4F1B5C1D5F1B6C1D6F113
:1011F000B7C1D7F1B8C1D8F1B9C1D9F10101555181
:101200005B2756515C23E86A5D230E2E10EF09F030
:101210005CC157F15DC158F15B6B5C6B5D6B078E18
:1012200012EF09F002C0E0FF005001C0D8FF10002B
:10123000A6B218EF09F00CC0A9FF0BC0A8FFA69E2C
:10124000A69CA684F29E550EA76EAA0EA76EA68235
:10125000F28EA694A6B22AEF09F00C2A1200A96E0B
:10126000A69EA69CA680A8500C2A120004012C0E53
:10127000826F4FEC0BF0D9EC23F00C502FEC09F0FF
:10128000E8CF00F10C502FEC09F0E8CF01F101AFED
:101290004FEF09F00101FF0E026FFF0E036F62ECCA
:1012A00023F029675BEF09F00401200E826F4FECF9
:1012B0000BF060EF09F004012D0E826F4FEC0BF084
:1012C0006CEC21F0120015941596076A0F6A106AEB
:1012D000116A126A136A166A0F010E0EC16E860E2B
:1012E000C06E030EC26E0F01896A110E926E080E57
:1012F0008A6EF10E936E8B6A800E946EF18E8A84E4
:101300008B86FC0E2FEC09F0E8CF0BF00BA01180C0
:101310000BA211820BA411840BA81188C90E2FEC0B
:1013200009F0E8CF1AF0CA0E2FEC09F0E8CF1BF055
:10133000CB0E2FEC09F0E8CF1CF0CC0E2FEC09F00F
:10134000E8CF1DF0FB0E2FEC09F0E8CF37F0CE0E02
:101350002FEC09F0E8CF14F0CD0E2FEC09F0E8CF18
:1013600036F01F6A206A0E6A01015B6B5C6B5D6B75
:10137000576B586BF29A0101476B486B496B4A6B8C
:101380004B6B4C6B4D6B4E6B4F6B506B516B526B91
:10139000456B466BD76AD66A0F01280ED56EF28A66
:1013A0009D90B00ECD6E01015E6B5F6B606B616BEB
:1013B000626B636B646B656B666B676B686B696BA9
:1013C000536B546BCF6ACE6A0F9A0F9C0F9E9D8011
:1013D000760ECA6E9D8202013C0E006FCC6A160E1C
:1013E0002FEC09F0E8CF00F1170E2FEC09F0E8CF51
:1013F00001F1180E2FEC09F0E8CF02F1190E2FECD5
:1014000009F0E8CF03F1010103AF21EF0AF0D9ECB5
:1014100023F0160E0C6E00C10BF018EC09F0170E3D
:101420000C6E01C10BF018EC09F0180E0C6E02C125
:101430000BF018EC09F0190E0C6E03C10BF018EC50
:1014400009F000C18EF101C18FF102C190F103C119
:1014500091F100C192F101C193F102C194F103C174
:1014600095F11A0E2FEC09F0E8CF00F11B0E2FECCE
:1014700009F0E8CF01F11C0E2FEC09F0E8CF02F1E2
:101480001D0E2FEC09F0E8CF03F1010103AF77EF58
:101490000AF0D9EC23F01A0E0C6E00C10BF018EC18
:1014A00009F01B0E0C6E01C10BF018EC09F01C0EBC
:1014B0000C6E02C10BF018EC09F01D0E0C6E03C18E
:1014C0000BF018EC09F01A0E2FEC09F0E8CF00F140
:1014D0001B0E2FEC09F0E8CF01F11C0E2FEC09F0E8
:1014E000E8CF02F11D0E2FEC09F0E8CF03F100C1A7
:1014F00096F101C197F102C198F103C199F1240E4F
:10150000AC6E900EAB6E240EAC6E080EB86E000E74
:10151000B06E1F0EAF6E0401806B816B0F01900ED9
:10152000AB6E0F019D8A0301806B816BC26B8B9246
:1015300007900001F28EF28C07B01AEF20F00FB086
:10154000EFEF18F010BEEFEF18F012B8EFEF18F051
:101550000301805181197F0BD8B41AEF20F013EEEC
:1015600000F081517F0BE126812BE7CFE8FFE00BF4
:10157000D8B41AEF20F023EE82F0C2513F0BD926E7
:10158000E7CFDFFFC22BDF50780AD8A41AEF20F094
:10159000078092C100F193C101F194C102F195C19C
:1015A00003F10101040E046F000E056F000E066FBB
:1015B000000E076FC4EC22F000AFE8EF0AF0010163
:1015C000030E926F000E936F000E946F000E956FD6
:1015D00003018251720AD8B470EF18F08251520A96
:1015E000D8B470EF18F08251750AD8B470EF18F0C3
:1015F0008251680AD8B463EF0BF08251630AD8B401
:10160000D4EF1CF08251690AD8B43DEF13F0825137
:101610007A0AD8B450EF14F08251490AD8B462EF74
:1016200012F08251500AD8B480EF11F08251700A42
:10163000D8B4C3EF11F08251540AD8B4EEEF11F0D0
:101640008251740AD8B434EF12F08251410AD8B4EE
:1016500068EF0CF082514B0AD8B465EF0BF0825161
:101660006D0AD8B4D8EF10F082514D0AD8B4F1EF1A
:1016700010F08251730AD8B4A0EF17F08251530AC8
:10168000D8B405EF18F08251660AD8B4C3EF12F04F
:101690008251590AD8B429EF10F00BEF1DF0040164
:1016A00014EE00F080517F0BE12682C4E7FF802B0F
:1016B000120004010D0E826F4FEC0BF00A0E826FC8
:1016C0004FEC0BF0120009EF1DF004014B0E826F7E
:1016D0004FEC0BF004012C0E826F4FEC0BF081B835
:1016E00002D036B630D003018351430AD8B4AAEFF2
:1016F0000BF003018351630AD8B4ACEF0BF0030184
:101700008351520AD8B4AEEF0BF003018351720A31
:10171000D8B4B0EF0BF003018351470AD8B4B2EF4D
:101720000BF003018351670AD8B4B4EF0BF0030147
:101730008351540AD8B4B6EF0BF003018351740AF5
:10174000D8B426EF0CF003018351550AD8B4B8EF92
:101750000BF083D036807BD0369079D0368277D02C
:10176000369275D0368473D0369471D036866FD069
:1017700084C330F185C331F186C332F187C333F1BD
:101780000101296B27EC24F09EEC23F000C104F149
:1017900001C105F102C106F103C107F11AEC24F001
:1017A000200EF86EF76AF66A0900F5CF2CF10900F1
:1017B000F5CF2DF10900F5CF2EF10900F5CF2FF16E
:1017C0000900F5CF30F10900F5CF31F10900F5CF6F
:1017D00032F10900F5CF33F10101296B27EC24F038
:1017E0009EEC23F0C4EC22F001010067FFEF0BF048
:1017F0000167FFEF0BF00267FFEF0BF0036701D00B
:1018000025D004014E0E826F4FEC0BF004016F0ED9
:10181000826F4FEC0BF004014D0E826F4FEC0BF01A
:101820000401610E826F4FEC0BF00401740E826FA5
:101830004FEC0BF00401630E826F4FEC0BF00401D0
:10184000680E826F4FEC0BF009EF1DF03696CD0E4F
:101850000C6E36C00BF018EC09F0CD0E2FEC09F031
:10186000E8CF36F036B006D00401630E826F4FEC3D
:101870000BF005D00401430E826F4FEC0BF036B233
:1018800006D00401720E826F4FEC0BF005D00401FC
:10189000520E826F4FEC0BF036B406D00401670E87
:1018A000826F4FEC0BF005D00401470E826F4FECB6
:1018B0000BF036B606D00401740E826F4FEC0BF0BD
:1018C00005D00401540E826F4FEC0BF009EF1DF0B0
:1018D0000401410E826F4FEC0BF003018351310A7A
:1018E000D8B449EF0FF003018351320AD8B479EF2D
:1018F0000EF003018351330AD8B402EF0EF0030156
:101900008351340AD8B4F2EF0CF003018351350A45
:10191000D8B492EF0CF004013F0E826F4FEC0BF045
:1019200009EF1DF003018451300AD8B4B8EF0CF070
:1019300003018451310AD8B4BBEF0CF00301845188
:10194000650AD8B4ACEF0CF003018451640AD8B432
:10195000AFEF0CF0BCEF0CF03790B0EF0CF037802D
:10196000FB0E0C6E37C00BF018EC09F0BCEF0CF05E
:101970008B90BCEF0CF08B800401350E826F4FEC26
:101980000BF004012C0E826F4FEC0BF08BB0D0EFFC
:101990000CF00401300E826F4FEC0BF0D5EF0CF021
:1019A0000401310E826F4FEC0BF004012C0E826F9C
:1019B0004FEC0BF0FB0E2FEC09F0E8CF37F037A01F
:1019C000E9EF0CF00401640E826F4FEC0BF0EEEFC8
:1019D0000CF00401650E826F4FEC0BF0F0EF0CF091
:1019E00009EF1DF0CC0E2FEC09F0E8CF0BF004014D
:1019F0002C0E826F4FEC0BF003018451310AD8B4E6
:101A000016EF0DF003018451300AD8B418EF0DF031
:101A1000030184514D0AD8B422EF0DF00301845123
:101A2000540AD8B429EF0DF040EF0DF08A8401D0AC
:101A30008A940BAE04D00BAC02D00BBA21D0E00ECE
:101A40000B1218D01F0E0B168539E844E00B0B1251
:101A500011D0E00E0B161AEC24F085C332F186C3C8
:101A600033F10101296B27EC24F09EEC23F00051A7
:101A70001F0B0B12CC0E0C6E0BC00BF018EC09F008
:101A80000401340E826F4FEC0BF004012C0E826FB8
:101A90004FEC0BF0CC0E2FEC09F0E8CF1DF08AB420
:101AA00006D00401300E826F4FEC0BF005D004011C
:101AB000310E826F4FEC0BF004012C0E826F4FEC55
:101AC0000BF01D38E840070BE8CF82F40401300E1C
:101AD00082274FEC0BF004012C0E826F4FEC0BF0C1
:101AE000D9EC23F01D501F0BE8CF00F162EC23F07E
:101AF00032C182F40401300E82274FEC0BF033C167
:101B000082F40401300E82274FEC0BF004012C0EFE
:101B1000826F4FEC0BF0D9EC23F030C000F100AF36
:101B20000BD0FF0E016FFF0E026FFF0E036F04015B
:101B30002D0E826F4FEC0BF062EC23F031C182F47A
:101B40000401300E82274FEC0BF032C182F4040105
:101B5000300E82274FEC0BF033C182F40401300EBB
:101B600082274FEC0BF004012C0E826F4FEC0BF030
:101B7000D9EC23F02FC000F162EC23F031C182F4E4
:101B80000401300E82274FEC0BF032C182F40401C5
:101B9000300E82274FEC0BF033C182F40401300E7B
:101BA00082274FEC0BF004012C0E826F4FEC0BF0F0
:101BB000D9EC23F031C000F100AF0BD0FF0E016F64
:101BC000FF0E026FFF0E036F04012D0E826F4FECAC
:101BD0000BF062EC23F031C182F40401300E822755
:101BE0004FEC0BF032C182F40401300E82274FEC2F
:101BF0000BF033C182F40401300E82274FEC0BF05E
:101C000009EF1DF0CB0E2FEC09F0E8CF0BF004012B
:101C10002C0E826F4FEC0BF003018451450AD8B4AF
:101C200026EF0EF003018451440AD8B429EF0EF0D8
:101C300003018451300AD8B42CEF0EF00301845113
:101C4000310AD8B430EF0EF03BEF0EF00B9E35EFBB
:101C50000EF00B8E35EF0EF0FC0E0B1635EF0EF07E
:101C6000FC0E0B160B8035EF0EF0CB0E0C6E0BC07E
:101C70000BF018EC09F00401330E826F4FEC0BF0FF
:101C800004012C0E826F4FEC0BF0CB0E2FEC09F001
:101C9000E8CF1CF01CBE54EF0EF00401450E826F1D
:101CA0004FEC0BF059EF0EF00401440E826F4FEC35
:101CB0000BF004012C0E826F4FEC0BF00401300E80
:101CC000826F4FEC0BF004012C0E826F4FEC0BF087
:101CD0001CB072EF0EF00401300E826F4FEC0BF06F
:101CE00077EF0EF00401310E826F4FEC0BF009EF2D
:101CF0001DF0CA0E2FEC09F0E8CF0BF004012C0EFA
:101D0000826F4FEC0BF003018451450AD8B4B5EF54
:101D10000EF003018451440AD8B4B8EF0EF0030169
:101D200084514D0AD8B4C1EF0EF003018451410A29
:101D3000D8B4BBEF0EF003018451460AD8B4BEEF0D
:101D40000EF003018451560AD8B4C9EF0EF0030116
:101D50008451500AD8B4D4EF0EF003018451520AD2
:101D6000D8B4D7EF0EF0E0EF0EF00B9EDAEF0EF0E6
:101D70000B8EDAEF0EF00B9CDAEF0EF00B8CDAEF35
:101D80000EF0FC0E0B1685C3E8FF030B0B12DAEF07
:101D90000EF0C70E0B1685C3E8FF070BE846E846B2
:101DA000E8460B12DAEF0EF00B84DAEF0EF00B942C
:101DB000DAEF0EF0CA0E0C6E0BC00BF018EC09F047
:101DC000CA0E2FEC09F0E8CF1BF00401320E826F2F
:101DD0004FEC0BF004012C0E826F4FEC0BF01BBE8E
:101DE000F9EF0EF00401450E826F4FEC0BF0FEEFA1
:101DF0000EF00401440E826F4FEC0BF004012C0E28
:101E0000826F4FEC0BF01BC0E8FF030BE8CF82F4AE
:101E10000401300E82274FEC0BF004012C0E826F70
:101E20004FEC0BF01BBC1CEF0FF00401410E826F56
:101E30004FEC0BF021EF0FF00401460E826F4FECD8
:101E40000BF004012C0E826F4FEC0BF01BC0E8FF6F
:101E5000380BE842E842E842E8CF82F40401300E51
:101E600082274FEC0BF004012C0E826F4FEC0BF02D
:101E70001BB442EF0FF00401520E826F4FEC0BF0D7
:101E800047EF0FF00401500E826F4FEC0BF009EF9B
:101E90001DF0C90E2FEC09F0E8CF0BF004012C0E59
:101EA000826F4FEC0BF003018451450AD8B467EF01
:101EB0000FF003018451440AD8B46AEF0FF0030114
:101EC00084514D0AD8B46DEF0FF07BEF0FF00B9EED
:101ED00075EF0FF00B8E75EF0FF0F80E0B1685C334
:101EE000E8FF070B0B1275EF0FF0C90E0C6E0BC05D
:101EF0000BF018EC09F00401310E826F4FEC0BF07F
:101F000004012C0E826F4FEC0BF0C90E2FEC09F080
:101F1000E8CF1AF01ABE06D00401450E826F4FECCE
:101F20000BF005D00401440E826F4FEC0BF004015E
:101F30002C0E826F4FEC0BF01AC0E8FF070BE8CFB6
:101F400082F40401300E82274FEC0BF004012C0EBA
:101F5000826F4FEC0BF00780D9EC23F02BC0E8FF29
:101F6000003B00430043030B62EC23F033C182F4D7
:101F70000401300E82274FEC0BF004012C0E826F0F
:101F80004FEC0BF0D9EC23F02BC001F1019F019D28
:101F90002CC000F1010162EC23F02FC182F4040196
:101FA000300E82274FEC0BF030C182F40401300E6A
:101FB00082274FEC0BF031C182F40401300E8227EE
:101FC0004FEC0BF032C182F40401300E82274FEC4B
:101FD0000BF033C182F40401300E82274FEC0BF07A
:101FE00004012C0E826F4FEC0BF0D9EC23F02DC0C6
:101FF00001F12EC000F1D89001330033D8900133A5
:102000000033010162EC23F02FC182F40401300E91
:1020100082274FEC0BF030C182F40401300E82278E
:102020004FEC0BF031C182F40401300E82274FECEB
:102030000BF032C182F40401300E82274FEC0BF01A
:1020400033C182F40401300E82274FEC0BF009EF0C
:102050001DF0FC0E2FEC09F0E8CF0BF003018351CB
:10206000520AD8B460EF10F003018351720AD8B459
:1020700063EF10F003018351500AD8B466EF10F0FB
:1020800003018351700AD8B469EF10F00301835142
:10209000550AD8B46CEF10F003018351750AD8B417
:1020A0006FEF10F003018351430AD8B478EF10F0BA
:1020B00003018351630AD8B47BEF10F084EF10F072
:1020C0000B907EEF10F00B807EEF10F00B927EEF06
:1020D00010F00B827EEF10F00B947EEF10F00B846B
:1020E0007EEF10F00B967EEF10F00B867EEF10F077
:1020F0000B987EEF10F00B887EEF10F0FC0E0C6E4C
:102100000BC00BF018EC09F00401590E826F4FEC74
:102110000BF01190119211941198FC0E2FEC09F014
:10212000E8CF0BF00BA011800BA211820BA411843D
:102130000BA8118811A0A4EF10F00401520E826FB9
:102140004FEC0BF0A9EF10F00401720E826F4FEC10
:102150000BF011A8B3EF10F00401430E826F4FECA7
:102160000BF0B8EF10F00401630E826F4FEC0BF030
:1021700011A2C2EF10F00401500E826F4FEC0BF071
:10218000C7EF10F00401700E826F4FEC0BF011A43A
:10219000D1EF10F00401550E826F4FEC0BF0D6EF2B
:1021A00010F00401750E826F4FEC0BF009EF1DF07B
:1021B00004016D0E826F4FEC0BF003018351300A66
:1021C000D8B430EF11F003018351310AD8B443EF92
:1021D00011F003018351320AD8B456EF11F00BEF1E
:1021E0001DF004014D0E826F4FEC0BF01AEC24F041
:1021F00084C331F185C332F186C333F10101296B08
:1022000027EC24F09EEC23F003018351300AD8B46C
:1022100018EF11F003018351310AD8B420EF11F007
:1022200003018351320AD8B428EF11F00BEF1DF0EF
:10223000FD0E0C6E00C10BF018EC09F030EF11F040
:10224000FE0E0C6E00C10BF018EC09F043EF11F01C
:10225000FF0E0C6E00C10BF018EC09F056EF11F0F8
:102260000401300E826F4FEC0BF004012C0E826FD4
:102270004FEC0BF0D9EC23F0FD0E2FEC09F0E8CF7A
:1022800000F167EF11F00401310E826F4FEC0BF09B
:1022900004012C0E826F4FEC0BF0D9EC23F0FE0EF4
:1022A0002FEC09F0E8CF00F167EF11F00401320ED6
:1022B000826F4FEC0BF0D9EC23F004012C0E826FEF
:1022C0004FEC0BF0FF0E2FEC09F0E8CF00F162ECC1
:1022D00023F031C182F40401300E82274FEC0BF061
:1022E00032C182F40401300E82274FEC0BF033C16F
:1022F00082F40401300E82274FEC0BF009EF1DF041
:1023000083C32AF184C32BF185C32CF186C32DF13D
:1023100087C32EF188C32FF189C330F18AC331F10D
:102320008BC332F18CC333F1010127EC24F09EEC16
:1023300023F0160E0C6E00C10BF018EC09F0170E0E
:102340000C6E01C10BF018EC09F0180E0C6E02C1F6
:102350000BF018EC09F0190E0C6E03C10BF018EC21
:1023600009F000C18EF101C18FF102C190F103C1EA
:1023700091F100C192F101C193F102C194F103C145
:1023800095F162EF12F083C32AF184C32BF185C368
:102390002CF186C32DF187C32EF188C32FF189C399
:1023A00030F18AC331F18BC332F18CC333F10101B7
:1023B00027EC24F09EEC23F000C18EF101C18FF1D7
:1023C00002C190F103C191F100C192F101C193F1F9
:1023D00002C194F103C195F162EF12F083C32AF1B7
:1023E00084C32BF185C32CF186C32DF187C32EF155
:1023F00088C32FF189C330F18AC331F18CC332F124
:102400008DC333F1010127EC24F09EEC23F0010190
:10241000000E046F000E056F010E066F000E076FB1
:10242000D5EC22F01A0E0C6E00C10BF018EC09F07E
:102430001B0E0C6E01C10BF018EC09F01C0E0C6E9B
:1024400002C10BF018EC09F01D0E0C6E03C10BF06D
:1024500018EC09F000C196F101C197F102C198F1A1
:1024600003C199F162EF12F083C32AF184C32BF107
:1024700085C32CF186C32DF187C32EF188C32FF1BC
:1024800089C330F18AC331F18CC332F18DC333F18A
:10249000010127EC24F09EEC23F00101000E046FF3
:1024A000000E056F010E066F000E076FD5EC22F0CF
:1024B00000C196F101C197F102C198F103C199F1F0
:1024C00062EF12F0160E2FEC09F0E8CF00F1170EB4
:1024D0002FEC09F0E8CF01F1180E2FEC09F0E8CF4E
:1024E00002F1190E2FEC09F0E8CF03F162EC23F0B2
:1024F00025EC21F00401730E826F4FEC0BF0040108
:102500002C0E826F4FEC0BF08EC100F18FC101F1E8
:1025100090C102F191C103F162EC23F025EC21F0AE
:102520000401730E826F4FEC0BF004012C0E826FCE
:102530004FEC0BF01A0E2FEC09F0E8CF00F11B0E58
:102540002FEC09F0E8CF01F11C0E2FEC09F0E8CFD9
:1025500002F11D0E2FEC09F0E8CF03F126EC1DF07F
:1025600004012C0E826F4FEC0BF096C100F197C165
:1025700001F198C102F199C103F126EC1DF059EC6B
:102580000BF00BEF1DF00401660E826F4FEC0BF0A9
:1025900003018351780AD8B4F0EF12F0030183519C
:1025A000430AD8B4F4EF12F003018351460AD8B4B9
:1025B000FDEF12F0030183B102D08B9601D08B8620
:1025C00083B302D08A9401D08A8484B102D08B9ADA
:1025D00001D08B8A84B302D08B9801D08B88138072
:1025E00000EC13F009EF1DF0149ECE0E0C6E14C01B
:1025F0000BF018EC09F0F0EF12F0148EF5EF12F07A
:1026000004012C0E826F4FEC0BF0300E8BB602D013
:10261000E89001D0E8808AB402D0E89201D0E88244
:10262000E8CF82F44FEC0BF004012C0E826F4FECDC
:102630000BF0300E8BBA02D0E89001D0E8808BB856
:1026400002D0E89201D0E882E8CF82F44FEC0BF0A0
:1026500004012C0E826F4FEC0BF014AE37EF13F029
:102660000401460E826F4FEC0BF03CEF13F00401B7
:10267000430E826F4FEC0BF012000401690E826F63
:102680004FEC0BF004012C0E826F4FEC0BF00101AC
:10269000040E006F000E016F000E026F000E036F3C
:1026A00062EC23F02CC182F40401300E82274FEC3F
:1026B0000BF02DC182F40401300E82274FEC0BF099
:1026C0002EC182F40401300E82274FEC0BF02FC193
:1026D00082F40401300E82274FEC0BF030C182F4FB
:1026E0000401300E82274FEC0BF031C182F404015B
:1026F000300E82274FEC0BF032C182F40401300E11
:1027000082274FEC0BF033C182F40401300E822794
:102710004FEC0BF004012C0E826F4FEC0BF001011B
:10272000040E006F000E016F000E026F000E036FAB
:1027300062EC23F02CC182F40401300E82274FECAE
:102740000BF02DC182F40401300E82274FEC0BF008
:102750002EC182F40401300E82274FEC0BF02FC102
:1027600082F40401300E82274FEC0BF030C182F46A
:102770000401300E82274FEC0BF031C182F40401CA
:10278000300E82274FEC0BF032C182F40401300E80
:1027900082274FEC0BF033C182F40401300E822704
:1027A0004FEC0BF004012C0E826F4FEC0BF001018B
:1027B0004F0E006F000E016F000E026F000E036FD0
:1027C00062EC23F02CC182F40401300E82274FEC1E
:1027D0000BF02DC182F40401300E82274FEC0BF078
:1027E0002EC182F40401300E82274FEC0BF02FC172
:1027F00082F40401300E82274FEC0BF030C182F4DA
:102800000401300E82274FEC0BF031C182F4040139
:10281000300E82274FEC0BF032C182F40401300EEF
:1028200082274FEC0BF033C182F40401300E822773
:102830004FEC0BF004012C0E826F4FEC0BF0200ECE
:10284000F86EF76AF66A04010900F5CF82F44FECDE
:102850000BF00900F5CF82F44FEC0BF00900F5CF37
:1028600082F44FEC0BF00900F5CF82F44FEC0BF043
:102870000900F5CF82F44FEC0BF00900F5CF82F49C
:102880004FEC0BF00900F5CF82F44FEC0BF0090090
:10289000F5CF82F44FEC0BF059EC0BF00BEF1DF081
:1028A0008351630AD8A409EF1DF08451610AD8A4AA
:1028B00009EF1DF085516C0AD8A409EF1DF086516F
:1028C000410A3FE08651440A1BE08651420AD8B4CF
:1028D000B4EF14F08651350AD8B495EF1EF0865146
:1028E000360AD8B4EAEF1EF08651370AD8B453EF4F
:1028F0001FF08651380AD8B4B1EF1FF009EF1DF070
:102900000798079A04017A0E826F4FEC0BF00401CE
:10291000780E826F4FEC0BF00401640E826F4FEC67
:102920000BF00401550E826F4FEC0BF09DEF14F08D
:1029300004014C0E826F4FEC0BF059EC0BF00BEFD7
:102940001DF00788079A04017A0E826F4FEC0BF096
:102950000401410E826F4FEC0BF00401610E826F97
:102960004FEC0BF091EF14F00798078A04017A0EF0
:10297000826F4FEC0BF00401420E826F4FEC0BF0B4
:102980000401610E826F4FEC0BF091EF14F0010126
:102990006667D2EF14F06767D2EF14F06867D2EF82
:1029A00014F0696716D001014F67DEEF14F050672D
:1029B000DEEF14F05167DEEF14F052670AD0010128
:1029C000000E006F000E016F000E026F000E036F0D
:1029D000120011B80AD00101620E046F010E056FDA
:1029E000000E066F000E076F09D00101A70E046FDD
:1029F000020E056F000E066F000E076F66C100F134
:102A000067C101F168C102F169C103F1C4EC22F0B0
:102A100003BF7BEF15F0119A119C0101000E046FAA
:102A2000A80E056F550E066F020E076F66C100F106
:102A300067C101F168C102F169C103F166C18AF1A0
:102A400067C18BF168C18CF169C18DF1C4EC22F0D2
:102A500003BF0BD00101000E8A6FA80E8B6F550EBD
:102A60008C6F020E8D6F118A119C0E0E2FEC09F0E7
:102A7000E8CF18F10F0E2FEC09F0E8CF19F1100E86
:102A80002FEC09F0E8CF1AF1110E2FEC09F0E8CF86
:102A90001BF10DEC22F08AC104F18BC105F18CC150
:102AA00006F18DC107F1C4EC22F00782D1EC21F0D0
:102AB0000DEC22F00792D1EC21F08AC100F18BC11C
:102AC00001F18CC102F18DC103F10792D1EC21F02B
:102AD000CC0E046FE00E056F870E066F050E076FB4
:102AE000C4EC22F000C118F101C119F102C11AF1C0
:102AF00003C11BF140D013AA80EF15F0138E139A77
:102B0000119C119A0101800E006F1A0E016F060EC2
:102B1000026F000E036F4FC104F150C105F151C1A6
:102B200006F152C107F1C4EC22F003AF05D0D9EC95
:102B300023F0118C119A12000E0E2FEC09F0E8CF41
:102B400018F10F0E2FEC09F0E8CF19F1100E2FEC51
:102B500009F0E8CF1AF1110E2FEC09F0E8CF1BF1C4
:102B60004FC100F150C101F151C102F152C103F155
:102B70000782D1EC21F018C100F119C101F11AC18D
:102B800002F11BC103F112000784BAC166F1BBC197
:102B900067F1BCC168F1BDC169F14BC14FF14CC1D6
:102BA00050F14DC151F14EC152F157C159F158C1C7
:102BB0005AF1079401016667E5EF15F06767E5EFE5
:102BC00015F06867E5EF15F0696716D001014F67EA
:102BD000F1EF15F05067F1EF15F05167F1EF15F0D7
:102BE00052670AD00101000E006F000E016F000E47
:102BF000026F000E036F120011B80AD00101620EBD
:102C0000046F010E056F000E066F000E076F09D0EE
:102C10000101A70E046F020E056F000E066F000E75
:102C2000076F66C100F167C101F168C102F169C1B6
:102C300003F1C4EC22F003BF7DEF16F00101000E9A
:102C4000046FA80E056F550E066F020E076F66C162
:102C500000F167C101F168C102F169C103F166C108
:102C60008AF167C18BF168C18CF169C18DF1C4EC47
:102C700022F003BF09D00101000E8A6FA80E8B6FEE
:102C8000550E8C6F020E8D6F0DEC22F000C104F119
:102C900001C105F102C106F103C107F1000E006F89
:102CA000A00E016F980E026F7B0E036FF5EC22F001
:102CB00000C118F101C119F102C11AF103C11BF1E0
:102CC000000E006FA00E016F980E026F7B0E036F57
:102CD0008AC104F18BC105F18CC106F18DC107F1E8
:102CE000F5EC22F018C104F119C105F11AC106F181
:102CF0001BC107F1C4EC22F012000101A80E006F05
:102D0000610E016F000E026F000E036F4FC104F1E0
:102D100050C105F151C106F152C107F1C4EC22F0D6
:102D200003AF0AD00101A80E006F610E016F000E03
:102D3000026F000E036F00D0C80E006FAF0E016F60
:102D4000000E026F000E036F4FC104F150C105F178
:102D500051C106F152C107F1D5EC22F012000784EF
:102D6000BAC166F1BBC167F1BCC168F1BDC169F10F
:102D70004BC14FF14CC150F14DC151F14EC152F117
:102D800057C159F158C15AF1079401016667D0EF54
:102D900016F06767D0EF16F06867D0EF16F0696736
:102DA00016D001014F67DCEF16F05067DCEF16F02C
:102DB0005167DCEF16F052670AD00101000E006F78
:102DC000000E016F000E026F000E036F120011B8AB
:102DD0000AD00101620E046F010E056F000E066F2E
:102DE000000E076F09D00101A70E046F020E056FD8
:102DF000000E066F000E076F66C100F167C101F19A
:102E000068C102F169C103F1C4EC22F003BF92EF83
:102E100017F00101000E046FA80E056F550E066F26
:102E2000020E076F66C100F167C101F168C102F1CE
:102E300069C103F166C18AF167C18BF168C18CF188
:102E400069C18DF1C4EC22F003BF09D00101000E6D
:102E50008A6FA80E8B6F550E8C6F020E8D6F010E50
:102E6000006F000E016F000E026F000E036F8AC12B
:102E700004F18BC105F18CC106F18DC107F1F5ECB0
:102E800022F018C104F119C105F11AC106F11BC1E4
:102E900007F162EC23F02AC182F40401300E82278C
:102EA0004FEC0BF02BC182F40401300E82274FEC63
:102EB0000BF02CC182F40401300E82274FEC0BF092
:102EC0002DC182F40401300E82274FEC0BF02EC18D
:102ED00082F40401300E82274FEC0BF02FC182F4F4
:102EE0000401300E82274FEC0BF030C182F4040154
:102EF000300E82274FEC0BF031C182F40401300E0A
:102F000082274FEC0BF032C182F40401300E82278D
:102F10004FEC0BF033C182F40401300E82274FECEA
:102F20000BF012004FC100F150C101F151C102F18B
:102F300052C103F1010162EC23F025EC21F01200F3
:102F40000401730E826F4FEC0BF004012C0E826FA4
:102F50004FEC0BF0078462C166F163C167F164C195
:102F600068F165C169F14BC14FF14CC150F14DC1E0
:102F700051F14EC152F157C159F158C15AF107945C
:102F8000C6EC17F059EC0BF00BEF1DF066C100F129
:102F900067C101F168C102F169C103F1010162EC8D
:102FA00023F025EC21F00401630E826F4FEC0BF04F
:102FB00004012C0E826F4FEC0BF04FC100F150C199
:102FC00001F151C102F152C103F1010162EC23F0A0
:102FD00025EC21F00401660E826F4FEC0BF004012A
:102FE0002C0E826F4FEC0BF0D9EC23F059C100F19D
:102FF0005AC101F1010162EC23F025EC21F004013A
:10300000740E826F4FEC0BF0120010820401530E0D
:10301000826F4FEC0BF004012C0E826F4FEC0BF023
:1030200083C32AF184C32BF185C32CF186C32DF110
:1030300087C32EF188C32FF189C330F18AC331F1E0
:103040008BC332F18CC333F1010127EC24F09EECE9
:1030500023F000C166F101C167F102C168F103C14B
:1030600069F18EC32AF18FC32BF190C32CF191C368
:103070002DF192C32EF193C32FF194C330F195C378
:1030800031F196C332F197C333F1010127EC24F0FB
:103090009EEC23F000C14FF101C150F102C151F18A
:1030A00003C152F11AEC24F099C32FF19AC330F105
:1030B0009BC331F19CC332F19DC333F1010127EC75
:1030C00024F09EEC23F000C159F101C15AF1C6EC85
:1030D00017F004012C0E826F4FEC0BF080EF18F00C
:1030E000118E1CA002D01CAE108C1BBE02D01BA4E3
:1030F000108E03018251520A02E10F8201D00F9219
:103100008251750A02E1108401D010948251550A4F
:1031100002E1108601D010968351310A03E1138237
:10312000138402D01392139403018351660A01E0C1
:1031300056D00401660E826F4FEC0BF004012C0E8A
:10314000826F4FEC0BF0C4EC15F062EC23F02AC157
:1031500082F40401300E82274FEC0BF02BC182F475
:103160000401300E82274FEC0BF02CC182F40401D5
:10317000300E82274FEC0BF02DC182F40401300E8B
:1031800082274FEC0BF02EC182F40401300E82270F
:103190004FEC0BF02FC182F40401300E82274FEC6C
:1031A0000BF030C182F40401300E82274FEC0BF09B
:1031B00031C182F40401300E82274FEC0BF032C192
:1031C00082F40401300E82274FEC0BF033C182F4FD
:1031D0000401300E82274FEC0BF009EF1DF011A017
:1031E00003D011A401D01084078410B259EF19F054
:1031F00010A43DEF19F0BAC166F1BBC167F1BCC1C3
:1032000068F1BDC169F1BEC16AF1BFC16BF1C0C156
:103210006CF1C1C16DF1C2C16EF1C3C16FF1C4C126
:1032200070F1C5C171F1C6C172F1C7C173F1C8C1F6
:1032300074F1C9C175F1CAC176F1CBC177F1CCC1C6
:1032400078F1CDC179F1CEC17AF1CFC17BF1D0C196
:103250007CF1D1C17DF1D2C17EF1D3C17FF1D4C166
:1032600080F1D5C181F1D6C182F1D7C183F1D8C136
:1032700084F1D9C185F145EF19F062C166F163C1EE
:1032800067F164C168F165C169F1BAC186F1BBC17A
:1032900087F1BCC188F1BDC189F14BC14FF14CC16F
:1032A00050F14DC151F14EC152F157C159F158C1C0
:1032B0005AF107940FA07BEF19F00101966768EFB0
:1032C00019F0976768EF19F0986768EF19F0996738
:1032D0006CEF19F07BEF19F0C7EC14F096C104F114
:1032E00097C105F198C106F199C107F1C4EC22F02C
:1032F00003BFCFEF1CF0C7EC14F00101000E046F08
:10330000000E056F010E066F000E076FF5EC22F040
:1033100011A02AD011A228D062EC23F0296701D095
:1033200005D004012D0E826F4FEC0BF030C182F4FA
:103330000401300E82274FEC0BF031C182F40401FE
:10334000300E82274FEC0BF032C182F40401300EB4
:1033500082274FEC0BF033C182F40401300E822738
:103360004FEC0BF059EC0BF012A8C5D012981DC011
:103370001EF01E3A1E42070E1E1600011E50000AC5
:10338000D8B447EF1AF000011E50010AD8B4D3EFA9
:1033900019F000011E50020AD8B4D1EF19F079EFEC
:1033A0001AF079EF1AF0D9EC23F02DC001F12EC0FC
:1033B00000F1D89001330033D8900133003301017C
:1033C000630E046F000E056F000E066F000E076F90
:1033D000F5EC22F0280E046F000E056F000E066F4C
:1033E000000E076FC4EC22F000C130F0D9EC23F0DE
:1033F0002BC001F1019F019D2CC000F10101A40E21
:10340000046F000E056F000E066F000E076FF5ECDF
:1034100022F000C12FF000C104F101C105F102C189
:1034200006F103C107F1640E006F000E016F000E7C
:10343000026F000E036FC4EC22F0050E046F000E45
:10344000056F000E066F000E076FF5EC22F000C14D
:1034500004F101C105F102C106F103C107F1D9EC84
:1034600023F030C000F1C4EC22F000C131F031C0D3
:10347000E8FF050F305C03E78A8479EF1AF031C06A
:10348000E8FF0A0F305C01E68A9479EF1AF000C178
:1034900024F101C125F102C126F103C127F1D9ECC4
:1034A00023F0DFEC23F01D501F0BE8CF00F10101EA
:1034B000640E046F000E056F000E066F000E076F9E
:1034C000D5EC22F024C104F125C105F126C106F195
:1034D00027C107F1C4EC22F003BF02D08A9401D0C7
:1034E0008A8424C100F125C101F126C102F127C15E
:1034F00003F10BEF1DF000C124F101C125F102C160
:1035000026F103C127F110AE4DD0109E00C108F185
:1035100001C109F102C10AF103C10BF162EC23F010
:1035200030C1E2F131C1E3F132C1E4F133C1E5F17F
:1035300008C100F109C101F10AC102F10BC103F197
:1035400001016C0E046F070E056F000E066F000E72
:10355000076FC4EC22F003BF04D00101550EE66FE3
:103560001CD008C100F109C101F10AC102F10BC16F
:1035700003F10101A40E046F060E056F000E066F25
:10358000000E076FC4EC22F003BF04D001017F0ED0
:10359000E66F03D00101FF0EE66F1F8E11AECFEF75
:1035A0001CF0119E24C100F125C101F126C102F1D8
:1035B00027C103F111A005D011A203D00FB0CFEFA6
:1035C0001CF010A4EBEF1AF00401750E826F4FECA3
:1035D0000BF0F0EF1AF00401720E826F4FEC0BF05B
:1035E00004012C0E826F4FEC0BF062EC23F0296784
:1035F000FFEF1AF00401200E826F02EF1BF00401AE
:103600002D0E826F4FEC0BF030C182F40401300EAE
:1036100082274FEC0BF031C182F40401300E822777
:103620004FEC0BF004012E0E826F4FEC0BF032C109
:1036300082F40401300E82274FEC0BF033C182F488
:103640000401300E82274FEC0BF004016D0E826FE7
:103650004FEC0BF004012C0E826F4FEC0BF04FC1BE
:1036600000F150C101F151C102F152C103F1010158
:1036700062EC23F025EC21F00401480E826F4FEC40
:103680000BF004017A0E826F4FEC0BF004012C0E4C
:10369000826F4FEC0BF066C100F167C101F168C1A8
:1036A00002F169C103F1010162EC23F025EC21F084
:1036B0000401630E826F4FEC0BF004012C0E826F3D
:1036C0004FEC0BF066C100F167C101F168C102F176
:1036D00069C103F101010A0E046F000E056F000EAF
:1036E000066F000E076FD5EC22F0000E046F120E6D
:1036F000056F000E066F000E076FF5EC22F062EC0E
:1037000023F02AC182F40401300E82274FEC0BF023
:103710002BC182F40401300E82274FEC0BF02CC138
:1037200082F40401300E82274FEC0BF02DC182F49D
:103730000401300E82274FEC0BF02EC182F40401FD
:10374000300E82274FEC0BF02FC182F40401300EB3
:1037500082274FEC0BF030C182F40401300E822737
:103760004FEC0BF004012E0E826F4FEC0BF031C1C9
:1037700082F40401300E82274FEC0BF032C182F448
:103780000401300E82274FEC0BF033C182F40401A8
:10379000300E82274FEC0BF00401730E826F4FEC5A
:1037A0000BF004012C0E826F4FEC0BF0D9EC23F0E0
:1037B00059C100F15AC101F135EC1EF000EC13F0D3
:1037C00014BEF9EF1BF08BBA02D0E89001D0E8806C
:1037D0008BB802D0E89201D0E882E82A030BE8B067
:1037E00002D08B9A01D08B8AE8B202D08B9801D09C
:1037F0008B8813A24BEF1CF004012C0E826F4FEC50
:103800000BF086C166F187C167F188C168F189C193
:1038100069F1C7EC14F00101000E046F000E056F92
:10382000010E066F000E076FF5EC22F062EC23F03C
:10383000296720EF1CF00401200E826F23EF1CF09B
:1038400004012D0E826F4FEC0BF030C182F40401A5
:10385000300E82274FEC0BF031C182F40401300EA0
:1038600082274FEC0BF004012E0E826F4FEC0BF011
:1038700032C182F40401300E82274FEC0BF033C1C9
:1038800082F40401300E82274FEC0BF004016D0E20
:10389000826F4FEC0BF003018351460A01E007D021
:1038A00004012C0E826F4FEC0BF0AFEC16F013A45A
:1038B0007EEF1CF004012C0E826F4FEC0BF013AC6A
:1038C0006CEF1CF00401500E826F4FEC0BF0139C58
:1038D0001398139A7EEF1CF013AE79EF1CF00401DD
:1038E000460E826F4FEC0BF0139E1398139A7EEFE7
:1038F0001CF00401530E826F4FEC0BF037B095EFC4
:103900001CF004012C0E826F4FEC0BF08BB090EF8B
:103910001CF00401440E826F4FEC0BF095EF1CF08D
:103920000401530E826F4FEC0BF00FB29BEF1CF0B3
:103930000FA0CDEF1CF004012C0E826F4FEC0BF0AA
:10394000200EF86EF76AF66A04010900F5CF82F4DA
:103950004FEC0BF00900F5CF82F44FEC0BF00900AF
:10396000F5CF82F44FEC0BF00900F5CF82F44FEC69
:103970000BF00900F5CF82F44FEC0BF00900F5CF06
:1039800082F44FEC0BF00900F5CF82F44FEC0BF012
:103990000900F5CF82F44FEC0BF059EC0BF00F90CF
:1039A000109E12980BEF1DF00401630E826F4FEC16
:1039B0000BF004012C0E826F4FEC0BF011EC1DF09C
:1039C00004012C0E826F4FEC0BF084EC1DF004010F
:1039D0002C0E826F4FEC0BF000EC1EF004012C0E4D
:1039E000826F4FEC0BF00101F80E006FCD0E016FEE
:1039F000660E026F030E036F26EC1DF004012C0E01
:103A0000826F4FEC0BF016EC1EF059EC0BF00BEF45
:103A10001DF059EC0BF00301C26B079010921AEFE6
:103A200020F0D8900E0E2FEC09F0E8CF00F10F0E29
:103A30002FEC09F0E8CF01F1100E2FEC09F0E8CFE0
:103A400002F1110E2FEC09F0E8CF03F10101000E95
:103A5000046F000E056F010E066F000E076FF5EC88
:103A600022F062EC23F02AC182F40401300E822796
:103A70004FEC0BF02BC182F40401300E82274FEC87
:103A80000BF02CC182F40401300E82274FEC0BF0B6
:103A90002DC182F40401300E82274FEC0BF02EC1B1
:103AA00082F40401300E82274FEC0BF02FC182F418
:103AB0000401300E82274FEC0BF030C182F4040178
:103AC000300E82274FEC0BF031C182F40401300E2E
:103AD00082274FEC0BF004012E0E826F4FEC0BF09F
:103AE00032C182F40401300E82274FEC0BF033C157
:103AF00082F40401300E82274FEC0BF004016D0EAE
:103B0000826F4FEC0BF01200120E2FEC09F0E8CF91
:103B100000F1130E2FEC09F0E8CF01F1140E2FEC99
:103B200009F0E8CF02F1150E2FEC09F0E8CF03F110
:103B300001010A0E046F000E056F000E066F000EE5
:103B4000076FD5EC22F0000E046F120E056F000E09
:103B5000066F000E076FF5EC22F062EC23F02AC12D
:103B600082F40401300E82274FEC0BF02BC182F45B
:103B70000401300E82274FEC0BF02CC182F40401BB
:103B8000300E82274FEC0BF02DC182F40401300E71
:103B900082274FEC0BF02EC182F40401300E8227F5
:103BA0004FEC0BF02FC182F40401300E82274FEC52
:103BB0000BF030C182F40401300E82274FEC0BF081
:103BC00004012E0E826F4FEC0BF031C182F4040120
:103BD000300E82274FEC0BF032C182F40401300E1C
:103BE00082274FEC0BF033C182F40401300E8227A0
:103BF0004FEC0BF00401730E826F4FEC0BF01200D0
:103C00000A0E2FEC09F0E8CF00F10B0E2FEC09F0B3
:103C1000E8CF01F10C0E2FEC09F0E8CF02F10D0E08
:103C20002FEC09F0E8CF03F135EF1EF0060E2FEC74
:103C300009F0E8CF00F1070E2FEC09F0E8CF01F111
:103C4000080E2FEC09F0E8CF02F1090E2FEC09F075
:103C5000E8CF03F135EF1EF00101D9EC23F0078422
:103C600057C100F158C101F107940101E80E046F3A
:103C7000800E056F000E066F000E076FD5EC22F068
:103C8000000E046F040E056F000E066F000E076F26
:103C9000F5EC22F0880E046F130E056F000E066F10
:103CA000000E076FC4EC22F00A0E046F000E056FC1
:103CB000000E066F000E076FF5EC22F062EC23F0A9
:103CC0000101296769EF1EF00401200E826F6CEF7D
:103CD0001EF004012D0E826F4FEC0BF030C182F408
:103CE0000401300E82274FEC0BF031C182F4040145
:103CF000300E82274FEC0BF032C182F40401300EFB
:103D000082274FEC0BF004012E0E826F4FEC0BF06C
:103D100033C182F40401300E82274FEC0BF0040112
:103D2000430E826F4FEC0BF0120087C32AF188C359
:103D30002BF189C32CF18AC32DF18BC32EF18CC3D7
:103D40002FF18DC330F18EC331F190C332F191C3A5
:103D500033F10101296B27EC24F09EEC23F00101E3
:103D6000000E046F000E056F010E066F000E076F48
:103D7000D5EC22F00E0E0C6E00C10BF018EC09F021
:103D80000F0E0C6E01C10BF018EC09F0100E0C6E4A
:103D900002C10BF018EC09F0110E0C6E03C10BF010
:103DA00018EC09F004017A0E826F4FEC0BF004015D
:103DB0002C0E826F4FEC0BF00401350E826F4FEC2E
:103DC0000BF004012C0E826F4FEC0BF011EC1DF088
:103DD0009DEF14F087C32AF188C32BF189C32CF11E
:103DE0008AC32DF18BC32EF18CC32FF18DC330F11B
:103DF0008EC331F190C332F191C333F10101296BCC
:103E000027EC24F09EEC23F0880E046F130E056F50
:103E1000000E066F000E076FC9EC22F0000E046F53
:103E2000040E056F000E066F000E076FD5EC22F032
:103E30000101E80E046F800E056F000E066F000E84
:103E4000076FF5EC22F00A0E0C6E00C10BF018ECB7
:103E500009F00B0E0C6E01C10BF018EC09F00C0E02
:103E60000C6E02C10BF018EC09F00D0E0C6E03C1C4
:103E70000BF018EC09F004017A0E826F4FEC0BF096
:103E800004012C0E826F4FEC0BF00401360E826F92
:103E90004FEC0BF004012C0E826F4FEC0BF000EC9A
:103EA0001EF09DEF14F087C32AF188C32BF189C35C
:103EB0002CF18AC32DF18BC32EF18CC32FF18DC34E
:103EC00030F18FC331F190C332F191C333F101016D
:103ED00027EC24F09EEC23F0000E046F120E056F09
:103EE000000E066F000E076FD5EC22F001010A0EDE
:103EF000046F000E056F000E066F000E076FF5ECE5
:103F000022F0120E0C6E00C10BF018EC09F0130E2B
:103F10000C6E01C10BF018EC09F0140E0C6E02C10E
:103F20000BF018EC09F0150E0C6E03C10BF018EC39
:103F300009F004017A0E826F4FEC0BF004012C0E95
:103F4000826F4FEC0BF00401370E826F4FEC0BF0D9
:103F500004012C0E826F4FEC0BF084EC1DF09DEFF2
:103F600014F087C32AF188C32BF189C32CF18AC3CB
:103F70002DF18BC32EF18CC32FF18DC330F18EC385
:103F800031F190C332F191C333F10101296B27EC78
:103F900024F09EEC23F0880E046F130E056F000EC4
:103FA000066F000E076FC9EC22F0000E046F040EBE
:103FB000056F000E066F000E076FD5EC22F00101B1
:103FC000E80E046F800E056F000E066F000E076F7F
:103FD000F5EC22F0060E0C6E00C10BF018EC09F0A7
:103FE000070E0C6E01C10BF018EC09F0080E0C6EF8
:103FF00002C10BF018EC09F0090E0C6E03C10BF0B6
:1040000018EC09F004017A0E826F4FEC0BF00401FA
:104010002C0E826F4FEC0BF00401380E826F4FECC8
:104020000BF004012C0E826F4FEC0BF016EC1EF01F
:104030009DEF14F007A88DEF20F00101800E006FB6
:104040001A0E016F060E026F000E036F4BC104F1D2
:104050004CC105F14DC106F14EC107F1C4EC22F08F
:1040600003BFD3EF20F01FEC21F04BC100F14CC196
:1040700001F14DC102F14EC103F10782D1EC21F0F3
:1040800018C104F119C105F11AC106F11BC107F1EC
:10409000F80E006FCD0E016F660E026F030E036FF8
:1040A000C4EC22F00E0E0C6E00C10BF018EC09F0FF
:1040B0000F0E0C6E01C10BF018EC09F0100E0C6E17
:1040C00002C10BF018EC09F0110E0C6E03C10BF0DD
:1040D00018EC09F007840101D9EC23F057C100F175
:1040E00058C101F107940A0E0C6E00C10BF018ECD8
:1040F00009F00B0E0C6E01C10BF018EC09F00C0E60
:104100000C6E02C10BF018EC09F00D0E0C6E03C121
:104110000BF018EC09F0D3EF20F007AAD3EF20F052
:1041200007840101D9EC23F057C100F158C101F116
:104130000794060E0C6E00C10BF018EC09F0070E88
:104140000C6E01C10BF018EC09F0080E0C6E02C1E8
:104150000BF018EC09F0090E0C6E03C10BF018EC13
:1041600009F0078462C100F163C101F164C102F189
:1041700065C103F10794120E0C6E00C10BF018EC30
:1041800009F0130E0C6E01C10BF018EC09F0140EBF
:104190000C6E02C10BF018EC09F0150E0C6E03C189
:1041A0000BF018EC09F00798079A04018051811967
:1041B0007F0B0DE09EA8FED714EE00F081517F0B1F
:1041C000E126E750812B0F01AD6ED5EF20F09CEF7B
:1041D0000AF018C100F119C101F11AC102F11BC1A5
:1041E00003F1000E046F000E056F010E066F000E46
:1041F000076FF5EC22F029A114EF21F02051D8B47B
:1042000014EF21F018C100F119C101F11AC102F136
:104210001BC103F1000E046F000E056F0A0E066F3E
:10422000000E076FF5EC22F012000101045100139B
:104230000551011306510213075103131200010126
:10424000186B196B1A6B1B6B12002AC182F40401E4
:10425000300E82274FEC0BF02BC182F40401300E9C
:1042600082274FEC0BF02CC182F40401300E822720
:104270004FEC0BF02DC182F40401300E82274FEC7D
:104280000BF02EC182F40401300E82274FEC0BF0AC
:104290002FC182F40401300E82274FEC0BF030C1A5
:1042A00082F40401300E82274FEC0BF031C182F40E
:1042B0000401300E82274FEC0BF032C182F404016E
:1042C000300E82274FEC0BF033C182F40401300E24
:1042D00082274FEC0BF012002FC182F40401300E44
:1042E00082274FEC0BF030C182F40401300E82279C
:1042F0004FEC0BF031C182F40401300E82274FECF9
:104300000BF032C182F40401300E82274FEC0BF027
:1043100033C182F40401300E82274FEC0BF01200FF
:10432000060E216E060E226E060E236E212E96EFCD
:1043300021F0222E96EF21F0232E96EF21F08B8490
:10434000020E216E020E226E020E236E212EA6EFA9
:1043500021F0222EA6EF21F0232EA6EF21F08B9440
:104360001200FF0E226E22C023F0030E216E8B84FA
:10437000212EB7EF21F0030E216E232EB7EF21F08F
:104380008B9422C023F0030E216E212EC5EF21F065
:10439000030E216E233EC5EF21F0222EB3EF21F054
:1043A00012000101005305E1015303E1025301E151
:1043B000002B94EC22F0D9EC23F03951006F3A51E4
:1043C000016F420E046F4B0E056F000E066F000E5C
:1043D000076FD5EC22F000C104F101C105F102C163
:1043E00006F103C107F118C100F119C101F11AC1A9
:1043F00002F11BC103F107B202EF22F0C9EC22F077
:1044000004EF22F0C4EC22F000C118F101C119F14F
:1044100002C11AF103C11BF11200D9EC23F059C1FA
:1044200000F15AC101F1060E2FEC09F0E8CF04F1BA
:10443000070E2FEC09F0E8CF05F1080E2FEC09F07C
:10444000E8CF06F1090E2FEC09F0E8CF07F1C4EC34
:1044500022F000C124F101C125F102C126F103C1FE
:1044600027F1290E046F000E056F000E066F000E77
:10447000076FD5EC22F0EE0E046F430E056F000EB1
:10448000066F000E076FC9EC22F024C104F125C1AC
:1044900005F126C106F127C107F1D5EC22F000C1D4
:1044A0001CF101C11DF102C11EF103C11FF1120E69
:1044B0002FEC09F0E8CF04F1130E2FEC09F0E8CF50
:1044C00005F1140E2FEC09F0E8CF06F1150E2FECD4
:1044D00009F0E8CF07F10D0E006F000E016F000E1E
:1044E000026F000E036FD5EC22F0180E046F000E61
:1044F000056F000E066F000E076FF5EC22F01CC171
:1045000004F11DC105F11EC106F11FC107F1C9EC7F
:1045100022F06A0E046F2A0E056F000E066F000E61
:10452000076FC4EC22F01200BF0EFA6E200E3A6F35
:10453000396BD8900037013702370337D8B0A5EF71
:1045400022F03A2F9AEF22F039073A070353D8B4F2
:1045500012000331070B80093F6F03390F0B010F66
:10456000396F80EC5FF0406F390580EC5FF0405DA3
:10457000405F396B3F33D8B0392739333FA9BAEFA1
:1045800022F04051392712000101FEEC23F0D8B08F
:104590001200010103510719346FC1EC23F0D890C8
:1045A0000751031934AF800F12000101346BE5ECA1
:1045B00023F0D8A0FBEC23F0D8B01200D0EC23F00D
:1045C000D9EC23F01F0E366F11EC24F00B35D8B068
:1045D000C1EC23F0D8A00335D8B01200362FE4EF99
:1045E00022F034B1E8EC23F012000101346B0451E5
:1045F0000511061107110008D8A0E5EC23F0D8A09A
:10460000FBEC23F0D8B01200086B096B0A6B0B6B44
:1046100011EC24F01F0E366F11EC24F007510B5DE6
:10462000D8A41FEF23F006510A5DD8A41FEF23F092
:104630000551095DD8A41FEF23F00451085DD8A0EF
:1046400032EF23F00451085F0551D8A0053D095F02
:104650000651D8A0063D0A5F0751D8A0073D0B5F61
:10466000D8900081362F0CEF23F034B1E8EC23F022
:10467000346BE5EC23F0D89015EC24F007510B5D7A
:10468000D8A44FEF23F006510A5DD8A44FEF23F0D2
:104690000551095DD8A44FEF23F00451085DD8A05F
:1046A0005EEF23F0003F5EEF23F0013F5EEF23F06B
:1046B000023F5EEF23F0032BD8B4120034B1E8ECD4
:1046C00023F012000101346BE5EC23F0D8B01200A6
:1046D0001AEC24F0200E366F00370137023703370B
:1046E00011EE33F00A0E376FE7360A0EE75CD8B0EA
:1046F000E76EE552372F74EF23F0362F6CEF23F07F
:1047000034B12981D89012001AEC24F0200E366FB3
:10471000003701370237033711EE33F00A0E376FD7
:10472000E7360A0EE75CD8B0E76EE552372F90EF18
:1047300023F0362F88EF23F0D890120001010A0EE3
:10474000346F200E366F11EE29F03451376F0A0E98
:10475000D890E652D8B0E726E732372FA9EF23F0FA
:104760000333023301330033362FA3EF23F0E75036
:10477000FF0FD8A00335D8B0120029B1E8EC23F020
:104780001200045100270551D8B0053D01270651FC
:10479000D8B0063D02270751D8B0073D03271200C5
:1047A0000051086F0151096F02510A6F03510B6FDD
:1047B00012000101006B016B026B036B120001011F
:1047C000046B056B066B076B12000335D8A0120053
:1047D0000351800B001F011F021F031F003FF8EF52
:1047E00023F0013FF8EF23F0023FF8EF23F0032B13
:1047F000342B032512000735D8A012000751800B77
:10480000041F051F061F071F043F0EEF24F0053F7E
:104810000EEF24F0063F0EEF24F0072B342B072574
:1048200012000037013702370337083709370A37D4
:104830000B3712000101296B2A6B2B6B2C6B2D6B34
:104840002E6B2F6B306B316B326B336B12000101AF
:104850002A510F0B2A6F2B510F0B2B6F2C510F0B63
:104860002C6F2D510F0B2D6F2E510F0B2E6F2F51C3
:104870000F0B2F6F30510F0B306F31510F0B316F0A
:1048800032510F0B326F33510F0B336F120000C1D7
:1048900024F101C125F102C126F103C127F104C1B0
:1048A00000F105C101F106C102F107C103F124C104
:1048B00004F125C105F126C106F127C107F1120057
:10BF0000E844F926000C160C2B0C3F0C520C640C68
:10BF1000760C860C960CA50CB30CC10CCF0CDC0C6B
:06BF2000E80CF40C000C1B
:00000001FF
